:10000000031E080085015F30A000213084008001BC
:10001000840AA00B07282F2824208400073984068F
:100020000310840C840C840C041A841704128419A1
:10003000841684118A01820701340234043408349E
:10004000103420344034803407398A018207283440
:1000500029342A342B342C342D342E342F340730C9
:10006000B600193074217830B600FF3074210130A9
:100070006F21023064210330642104306421053093
:100080006F2108306F210130682105306821083068
:100090006821A1010130A00010212008C2219F2168
:1000A0003608A0000130B221031D5A287830A32160
:1000B00003194C282A30D321C2210030A821031D66
:1000C000E7282108C22101308F213608A1006430C1
:1000D00078212108C2211430AD21031D7128072188
:1000E000A1012A30D321C2210030A821031DE72815
:1000F0002B30D321C2210030A821031D5A281930EA
:1001000078212B30D321C2210030A821031D5A2889
:1001100005306C21A501A401013078212430C521CE
:1001200001308F212430CC212A30D321C22100304C
:10013000A821031DE7282430C5211130B9009430CF
:10014000AE21031D8C280130A0002B30D321C22109
:100150000130A821031DC3282A30D321C221003039
:10016000A821031DE728323078212008C2219F21D1
:100170003608A0000130B221031DC2288230A3211D
:100180000319A5285A28F920A501A4012A30D32152
:10019000C2210030A821031DE72801307821243036
:1001A000C52101308F212430CC212430C5211330CA
:1001B000B9008830A921031DE4282C30D321C221A5
:1001C0000130A821031DC62800215A2861210021E1
:1001D0002C30D321C2210130A821031DE82805308D
:1001E0006C210130B700F4307921053068215A289C
:1001F000DB2901306C2105306C2108306C21DB29B2
:10020000013068210530682108306821DB2905307C
:100210006C21643078210530682164307821DB2935
:1002200005306C2132307821053068213230782158
:1002300005306C2132307821053068213230782148
:1002400005306C2132307821053068213230782138
:1002500005306C2132307821053068213230782128
:1002600005306C2132307821053068213230782118
:1002700005306C2132307821053068213230782108
:1002800005306C21323078210530682132307821F8
:1002900005306C21323078210530682132307821E8
:1002A00005306C21323078210530682132307821D8
:1002B00005306C21323078210530682132307821C8
:1002C000DB290730862161290C2084178004DB2973
:1002D0000C20FF3A800571290C20800470290C2025
:1002E000FF3A84178005DB29840036088000DB296B
:1002F000B701B6009D2164003708360403190800D1
:10030000F730FF3E031D81299F217B298316F83892
:1003100081050F39810463000F308104DB29B901A5
:10032000B80036308400380880073908840F000090
:100330000318013E031C8007DB29B709B609B60A7A
:100340000319B70A0800B901B800B7210139DB2940
:10035000B901B800B7210239DB29B901B800B721CA
:100360000539DB29B901B800B7210439DB2939087F
:100370003702031DBF293808360203190234031C53
:1003800004340134B701B600DB2984000008B6004C
:10039000840A0008B700DB29840036088000840A3C
:1003A00037088000DB290D20BD000005841B3D06B9
:0C03B000031900340134831264000800BB
:02400E00DC3F95
:00000001FF
